Archive member included because of file (symbol)

c:/winavr/bin/../lib/gcc/avr/4.1.1/avr5\libgcc.a(_clear_bss.o)
                              default/wdt_drv.o (__do_clear_bss)

Allocating common symbols
Common symbol       size              file

endpoint_status     0x7               default/usb_standard_request.o
usb_configuration_nb
                    0x1               default/usb_standard_request.o
ret                 0x1               default/main.o
data_to_transfer    0x1               default/usb_standard_request.o
pbuffer             0x2               default/usb_standard_request.o

Discarded input sections

 .data          0x00000000        0x0 c:/winavr/bin/../lib/gcc/avr/4.1.1/../../../../avr/lib/avr5/crtusb1286.o
 .bss           0x00000000        0x0 c:/winavr/bin/../lib/gcc/avr/4.1.1/../../../../avr/lib/avr5/crtusb1286.o
 .stabstr       0x00000000        0x0 c:/winavr/bin/../lib/gcc/avr/4.1.1/../../../../avr/lib/avr5/crtusb1286.o
 .text          0x00000000        0x0 default/wdt_drv.o
 .data          0x00000000        0x0 default/wdt_drv.o
 .bss           0x00000000        0x0 default/wdt_drv.o
 .text.wdtdrv_interrupt_enable
                0x00000000        0x0 default/wdt_drv.o
 .text.wdtdrv_interrupt_reset_enable
                0x00000000        0x0 default/wdt_drv.o
 .text          0x00000000        0x0 default/usb_descriptors.o
 .data          0x00000000        0x0 default/usb_descriptors.o
 .bss           0x00000000        0x0 default/usb_descriptors.o
 .text          0x00000000        0x0 default/usb_device_task.o
 .data          0x00000000        0x0 default/usb_device_task.o
 .text          0x00000000        0x0 default/usb_drv.o
 .data          0x00000000        0x0 default/usb_drv.o
 .bss           0x00000000        0x0 default/usb_drv.o
 .text.usb_select_enpoint_interrupt
                0x00000000        0x0 default/usb_drv.o
 .text.usb_send_packet
                0x00000000        0x0 default/usb_drv.o
 .text.usb_read_packet
                0x00000000        0x0 default/usb_drv.o
 .text.usb_halt_endpoint
                0x00000000        0x0 default/usb_drv.o
 .text          0x00000000        0x0 default/start_boot.o
 .bss           0x00000000        0x0 default/start_boot.o
 .text.goto_boot
                0x00000000        0x0 default/start_boot.o
 .text          0x00000000        0x0 default/main.o
 .data          0x00000000        0x0 default/main.o
 .bss           0x00000000        0x0 default/main.o
 .text          0x00000000        0x0 default/usb_specific_request.o
 .data          0x00000000        0x0 default/usb_specific_request.o
 .text          0x00000000        0x0 default/usb_standard_request.o
 .data          0x00000000        0x0 default/usb_standard_request.o
 .text.usb_generate_remote_wakeup
                0x00000000        0x0 default/usb_standard_request.o
 .text          0x00000000        0x0 default/usb_task.o
 .data          0x00000000        0x0 default/usb_task.o
 .text          0x00000000        0x0 default/stk_525.o
 .data          0x00000000        0x0 default/stk_525.o
 .bss           0x00000000        0x0 default/stk_525.o
 .text          0x00000000        0x0 default/hid_task.o
 .data          0x00000000        0x0 default/hid_task.o
 .text          0x00000000        0x0 default/twimaster.o
 .data          0x00000000        0x0 default/twimaster.o
 .bss           0x00000000        0x0 default/twimaster.o
 .text.i2c_start_wait
                0x00000000        0x0 default/twimaster.o
 .text.i2c_rep_start
                0x00000000        0x0 default/twimaster.o
 .text.i2c_readAck
                0x00000000        0x0 default/twimaster.o
 .text.i2c_readNak
                0x00000000        0x0 default/twimaster.o
 .text          0x00000000        0x0 default/scheduler.o
 .data          0x00000000        0x0 default/scheduler.o
 .bss           0x00000000        0x0 default/scheduler.o
 .text.scheduler_empty_fct
                0x00000000        0x0 default/scheduler.o
 .text          0x00000000        0x0 c:/winavr/bin/../lib/gcc/avr/4.1.1/avr5\libgcc.a(_clear_bss.o)
 .data          0x00000000        0x0 c:/winavr/bin/../lib/gcc/avr/4.1.1/avr5\libgcc.a(_clear_bss.o)
 .bss           0x00000000        0x0 c:/winavr/bin/../lib/gcc/avr/4.1.1/avr5\libgcc.a(_clear_bss.o)
 .text.libgcc   0x00000000        0x0 c:/winavr/bin/../lib/gcc/avr/4.1.1/avr5\libgcc.a(_clear_bss.o)

Memory Configuration

Name             Origin             Length             Attributes
text             0x00000000         0x00020000         xr
data             0x00800060         0x0000ffa0         rw !x
eeprom           0x00810000         0x00010000         rw !x
*default*        0x00000000         0xffffffff

Linker script and memory map

Address of section .data set to 0x800100
LOAD c:/winavr/bin/../lib/gcc/avr/4.1.1/../../../../avr/lib/avr5/crtusb1286.o
LOAD default/wdt_drv.o
LOAD default/usb_descriptors.o
LOAD default/usb_device_task.o
LOAD default/usb_drv.o
LOAD default/start_boot.o
LOAD default/main.o
LOAD default/usb_specific_request.o
LOAD default/usb_standard_request.o
LOAD default/usb_task.o
LOAD default/stk_525.o
LOAD default/hid_task.o
LOAD default/twimaster.o
LOAD default/scheduler.o
LOAD c:/winavr/bin/../lib/gcc/avr/4.1.1/avr5\libgcc.a
LOAD c:/winavr/bin/../lib/gcc/avr/4.1.1/../../../../avr/lib/avr5\libc.a
LOAD c:/winavr/bin/../lib/gcc/avr/4.1.1/avr5\libgcc.a

.hash
 *(.hash)

.dynsym
 *(.dynsym)

.dynstr
 *(.dynstr)

.gnu.version
 *(.gnu.version)

.gnu.version_d
 *(.gnu.version_d)

.gnu.version_r
 *(.gnu.version_r)

.rel.init
 *(.rel.init)

.rela.init
 *(.rela.init)

.rel.text
 *(.rel.text)
 *(.rel.text.*)
 *(.rel.gnu.linkonce.t*)

.rela.text
 *(.rela.text)
 *(.rela.text.*)
 *(.rela.gnu.linkonce.t*)

.rel.fini
 *(.rel.fini)

.rela.fini
 *(.rela.fini)

.rel.rodata
 *(.rel.rodata)
 *(.rel.rodata.*)
 *(.rel.gnu.linkonce.r*)

.rela.rodata
 *(.rela.rodata)
 *(.rela.rodata.*)
 *(.rela.gnu.linkonce.r*)

.rel.data
 *(.rel.data)
 *(.rel.data.*)
 *(.rel.gnu.linkonce.d*)

.rela.data
 *(.rela.data)
 *(.rela.data.*)
 *(.rela.gnu.linkonce.d*)

.rel.ctors
 *(.rel.ctors)

.rela.ctors
 *(.rela.ctors)

.rel.dtors
 *(.rel.dtors)

.rela.dtors
 *(.rela.dtors)

.rel.got
 *(.rel.got)

.rela.got
 *(.rela.got)

.rel.bss
 *(.rel.bss)

.rela.bss
 *(.rela.bss)

.rel.plt
 *(.rel.plt)

.rela.plt
 *(.rela.plt)

.text           0x00000000     0x1046
 *(.vectors)
 .vectors       0x00000000       0x98 c:/winavr/bin/../lib/gcc/avr/4.1.1/../../../../avr/lib/avr5/crtusb1286.o
                0x00000000                __vectors
                0x00000000                __vector_default
 *(.vectors)
 *(.progmem.gcc*)
 *(.progmem*)
 .progmem.data  0x00000098       0xa2 default/usb_descriptors.o
                0x00000101                usb_user_language_id
                0x00000098                usb_dev_desc
                0x000000df                usb_user_product_string_descriptor
                0x000000d3                usb_user_manufacturer_string_descriptor
                0x00000105                usb_hid_report_descriptor
                0x000000aa                usb_conf_desc
                0x0000013a                . = ALIGN (0x2)
                0x0000013a                __trampolines_start = .
 *(.trampolines)
 .trampolines   0x0000013a        0x0 linker stubs
 *(.trampolines*)
                0x0000013a                __trampolines_end = .
 *(.jumptables)
 *(.jumptables*)
 *(.lowtext)
 *(.lowtext*)
                0x0000013a                __ctors_start = .
 *(.ctors)
                0x0000013a                __ctors_end = .
                0x0000013a                __dtors_start = .
 *(.dtors)
                0x0000013a                __dtors_end = .
 SORT(*)(.ctors)
 SORT(*)(.dtors)
 *(.init0)
 .init0         0x0000013a        0x0 c:/winavr/bin/../lib/gcc/avr/4.1.1/../../../../avr/lib/avr5/crtusb1286.o
                0x0000013a                __init
 *(.init0)
 *(.init1)
 *(.init1)
 *(.init2)
 .init2         0x0000013a        0xc c:/winavr/bin/../lib/gcc/avr/4.1.1/../../../../avr/lib/avr5/crtusb1286.o
 *(.init2)
 *(.init3)
 .init3         0x00000146       0x18 default/main.o
                0x00000146                __low_level_init
 *(.init3)
 *(.init4)
 .init4         0x0000015e       0x1a c:/winavr/bin/../lib/gcc/avr/4.1.1/../../../../avr/lib/avr5/crtusb1286.o
                0x0000015e                __do_copy_data
 .init4         0x00000178       0x10 c:/winavr/bin/../lib/gcc/avr/4.1.1/avr5\libgcc.a(_clear_bss.o)
                0x00000178                __do_clear_bss
 *(.init4)
 *(.init5)
 *(.init5)
 *(.init6)
 *(.init6)
 *(.init7)
 *(.init7)
 *(.init8)
 *(.init8)
 *(.init9)
 .init9         0x00000188        0x2 c:/winavr/bin/../lib/gcc/avr/4.1.1/../../../../avr/lib/avr5/crtusb1286.o
 *(.init9)
 *(.text)
 .text          0x0000018a        0x2 c:/winavr/bin/../lib/gcc/avr/4.1.1/../../../../avr/lib/avr5/crtusb1286.o
                0x0000018a                __vector_22
                0x0000018a                __vector_28
                0x0000018a                __vector_1
                0x0000018a                __vector_32
                0x0000018a                __vector_34
                0x0000018a                __vector_24
                0x0000018a                __vector_12
                0x0000018a                __bad_interrupt
                0x0000018a                __vector_6
                0x0000018a                __vector_31
                0x0000018a                __vector_35
                0x0000018a                __vector_3
                0x0000018a                __vector_23
                0x0000018a                __vector_30
                0x0000018a                __vector_25
                0x0000018a                __vector_11
                0x0000018a                __vector_13
                0x0000018a                __vector_17
                0x0000018a                __vector_19
                0x0000018a                __vector_7
                0x0000018a                __vector_27
                0x0000018a                __vector_5
                0x0000018a                __vector_33
                0x0000018a                __vector_37
                0x0000018a                __vector_4
                0x0000018a                __vector_9
                0x0000018a                __vector_2
                0x0000018a                __vector_21
                0x0000018a                __vector_15
                0x0000018a                __vector_36
                0x0000018a                __vector_29
                0x0000018a                __vector_8
                0x0000018a                __vector_26
                0x0000018a                __vector_14
                0x0000018a                __vector_16
                0x0000018a                __vector_18
                0x0000018a                __vector_20
                0x0000018c                . = ALIGN (0x2)
 *(.text.*)
 .text.wdtdrv_disable
                0x0000018c       0x20 default/wdt_drv.o
                0x0000018c                wdtdrv_disable
 .text.wdtdrv_enable
                0x000001ac       0x34 default/wdt_drv.o
                0x000001ac                wdtdrv_enable
 .text.usb_device_task_init
                0x000001e0       0x1c default/usb_device_task.o
                0x000001e0                usb_device_task_init
 .text.usb_start_device
                0x000001fc       0x36 default/usb_device_task.o
                0x000001fc                usb_start_device
 .text.usb_device_task
                0x00000232       0xa2 default/usb_device_task.o
                0x00000232                usb_device_task
 .text.usb_config_ep
                0x000002d4       0x38 default/usb_drv.o
                0x000002d4                usb_config_ep
 .text.usb_init_device
                0x0000030c       0x32 default/usb_drv.o
                0x0000030c                usb_init_device
 .text.start_boot_if_required
                0x0000033e       0x36 default/start_boot.o
                0x0000033e                start_boot_if_required
 .text.start_boot
                0x00000374       0x1e default/start_boot.o
                0x00000374                start_boot
 .text.main     0x00000392       0x20 default/main.o
                0x00000392                main
 .text.usb_user_interface_get
                0x000003b2        0x6 default/usb_specific_request.o
                0x000003b2                usb_user_interface_get
 .text.usb_user_interface_reset
                0x000003b8       0x4c default/usb_specific_request.o
                0x000003b8                usb_user_interface_reset
 .text.usb_user_get_descriptor
                0x00000404       0x48 default/usb_specific_request.o
                0x00000404                usb_user_get_descriptor
 .text.hid_get_report_descriptor
                0x0000044c       0xe8 default/usb_specific_request.o
                0x0000044c                hid_get_report_descriptor
 .text.usb_hid_set_report_ouput
                0x00000534       0x3c default/usb_specific_request.o
                0x00000534                usb_hid_set_report_ouput
 .text.usb_hid_set_idle
                0x00000570       0x52 default/usb_specific_request.o
                0x00000570                usb_hid_set_idle
 .text.usb_hid_get_idle
                0x000005c2       0x7e default/usb_specific_request.o
                0x000005c2                usb_hid_get_idle
 .text.usb_hid_set_report_feature
                0x00000640       0x6a default/usb_specific_request.o
                0x00000640                usb_hid_set_report_feature
 .text.hid_get_hid_descriptor
                0x000006aa       0xe8 default/usb_specific_request.o
                0x000006aa                hid_get_hid_descriptor
 .text.usb_user_read_request
                0x00000792       0x62 default/usb_specific_request.o
                0x00000792                usb_user_read_request
 .text.usb_user_endpoint_init
                0x000007f4       0x26 default/usb_specific_request.o
                0x000007f4                usb_user_endpoint_init
 .text.usb_process_request
                0x0000081a      0x458 default/usb_standard_request.o
                0x0000081a                usb_process_request
 .text.__vector_10
                0x00000c72      0x1a0 default/usb_task.o
                0x00000c72                __vector_10
 .text.usb_task
                0x00000e12        0x4 default/usb_task.o
                0x00000e12                usb_task
 .text.usb_task_init
                0x00000e16       0x18 default/usb_task.o
                0x00000e16                usb_task_init
 .text.hid_task_init
                0x00000e2e       0x20 default/hid_task.o
                0x00000e2e                hid_task_init
 .text.hid_report_in
                0x00000e4e       0x7c default/hid_task.o
                0x00000e4e                hid_report_in
 .text.sof_action
                0x00000eca        0xc default/hid_task.o
                0x00000eca                sof_action
 .text.hid_report_out
                0x00000ed6       0xbc default/hid_task.o
                0x00000ed6                hid_report_out
 .text.hid_task
                0x00000f92        0xe default/hid_task.o
                0x00000f92                hid_task
 .text.i2c_init
                0x00000fa0        0xc default/twimaster.o
                0x00000fa0                i2c_init
 .text.i2c_start
                0x00000fac       0x54 default/twimaster.o
                0x00000fac                i2c_start
 .text.i2c_stop
                0x00001000       0x10 default/twimaster.o
                0x00001000                i2c_stop
 .text.i2c_write
                0x00001010       0x28 default/twimaster.o
                0x00001010                i2c_write
 .text.scheduler_tasks
                0x00001038        0x6 default/scheduler.o
                0x00001038                scheduler_tasks
 .text.scheduler_init
                0x0000103e        0x4 default/scheduler.o
                0x0000103e                scheduler_init
 .text.scheduler
                0x00001042        0x4 default/scheduler.o
                0x00001042                scheduler
                0x00001046                . = ALIGN (0x2)
 *(.fini9)
 *(.fini9)
 *(.fini8)
 *(.fini8)
 *(.fini7)
 *(.fini7)
 *(.fini6)
 *(.fini6)
 *(.fini5)
 *(.fini5)
 *(.fini4)
 *(.fini4)
 *(.fini3)
 *(.fini3)
 *(.fini2)
 *(.fini2)
 *(.fini1)
 *(.fini1)
 *(.fini0)
 *(.fini0)
                0x00001046                _etext = .

.data           0x00800100        0x2 load address 0x00001046
                0x00800100                PROVIDE (__data_start, .)
 *(.data)
 .data          0x00800100        0x2 default/start_boot.o
                0x00800100                start_bootloader
 *(.data*)
 *(.rodata)
 *(.rodata*)
 *(.gnu.linkonce.d*)
                0x00800102                . = ALIGN (0x2)
                0x00800102                _edata = .
                0x00800102                PROVIDE (__data_end, .)

.bss            0x00800102       0x15
                0x00800102                PROVIDE (__bss_start, .)
 *(.bss)
 .bss           0x00800102        0x2 default/usb_device_task.o
                0x00800103                usb_suspended
                0x00800102                usb_connected
 .bss           0x00800104        0x2 default/usb_specific_request.o
                0x00800104                jump_bootloader
                0x00800105                g_u8_report_rate
 .bss           0x00800106        0x1 default/usb_standard_request.o
                0x00800106                remote_wakeup_feature
 .bss           0x00800107        0x2 default/usb_task.o
                0x00800107                g_usb_event
 .bss           0x00800109        0x2 default/hid_task.o
                0x00800109                cpt_sof
                0x0080010a                g_last_joy
 *(.bss*)
 *(COMMON)
 COMMON         0x0080010b        0x1 default/main.o
                0x0080010b                ret
 COMMON         0x0080010c        0xb default/usb_standard_request.o
                0x0080010c                endpoint_status
                0x00800113                usb_configuration_nb
                0x00800114                data_to_transfer
                0x00800115                pbuffer
                0x00800117                PROVIDE (__bss_end, .)
                0x00001046                __data_load_start = LOADADDR (.data)
                0x00001048                __data_load_end = (__data_load_start + SIZEOF (.data))

.noinit         0x00800117        0x4
                0x00800117                PROVIDE (__noinit_start, .)
 *(.noinit*)
 .noinit        0x00800117        0x4 default/start_boot.o
                0x00800117                boot_key
                0x0080011b                PROVIDE (__noinit_end, .)
                0x0080011b                _end = .
                0x0080011b                PROVIDE (__heap_start, .)

.eeprom         0x00810000        0x0
 *(.eeprom*)
                0x00810000                __eeprom_end = .

.stab           0x00000000      0x408
 *(.stab)
 .stab          0x00000000      0x408 c:/winavr/bin/../lib/gcc/avr/4.1.1/../../../../avr/lib/avr5/crtusb1286.o

.stabstr        0x00000000       0x84
 *(.stabstr)
 .stabstr       0x00000000       0x84 c:/winavr/bin/../lib/gcc/avr/4.1.1/../../../../avr/lib/avr5/crtusb1286.o

.stab.excl
 *(.stab.excl)

.stab.exclstr
 *(.stab.exclstr)

.stab.index
 *(.stab.index)

.stab.indexstr
 *(.stab.indexstr)

.comment
 *(.comment)

.debug
 *(.debug)

.line
 *(.line)

.debug_srcinfo
 *(.debug_srcinfo)

.debug_sfnames
 *(.debug_sfnames)

.debug_aranges  0x00000000      0x2f8
 *(.debug_aranges)
 .debug_aranges
                0x00000000       0x40 default/wdt_drv.o
 .debug_aranges
                0x00000040       0x38 default/usb_device_task.o
 .debug_aranges
                0x00000078       0x50 default/usb_drv.o
 .debug_aranges
                0x000000c8       0x38 default/start_boot.o
 .debug_aranges
                0x00000100       0x30 default/main.o
 .debug_aranges
                0x00000130       0x78 default/usb_specific_request.o
 .debug_aranges
                0x000001a8       0x30 default/usb_standard_request.o
 .debug_aranges
                0x000001d8       0x38 default/usb_task.o
 .debug_aranges
                0x00000210       0x48 default/hid_task.o
 .debug_aranges
                0x00000258       0x60 default/twimaster.o
 .debug_aranges
                0x000002b8       0x40 default/scheduler.o

.debug_pubnames
                0x00000000      0x6c0
 *(.debug_pubnames)
 .debug_pubnames
                0x00000000       0x75 default/wdt_drv.o
 .debug_pubnames
                0x00000075       0xbf default/usb_descriptors.o
 .debug_pubnames
                0x00000134       0x78 default/usb_device_task.o
 .debug_pubnames
                0x000001ac       0x97 default/usb_drv.o
 .debug_pubnames
                0x00000243       0x6c default/start_boot.o
 .debug_pubnames
                0x000002af       0x38 default/main.o
 .debug_pubnames
                0x000002e7      0x163 default/usb_specific_request.o
 .debug_pubnames
                0x0000044a       0xb1 default/usb_standard_request.o
 .debug_pubnames
                0x000004fb       0x51 default/usb_task.o
 .debug_pubnames
                0x0000054c       0x88 default/hid_task.o
 .debug_pubnames
                0x000005d4       0x8d default/twimaster.o
 .debug_pubnames
                0x00000661       0x5f default/scheduler.o

.debug_info     0x00000000     0x23e0
 *(.debug_info)
 .debug_info    0x00000000      0x174 default/wdt_drv.o
 .debug_info    0x00000174      0x59a default/usb_descriptors.o
 .debug_info    0x0000070e      0x152 default/usb_device_task.o
 .debug_info    0x00000860      0x221 default/usb_drv.o
 .debug_info    0x00000a81      0x124 default/start_boot.o
 .debug_info    0x00000ba5      0x132 default/main.o
 .debug_info    0x00000cd7      0x7cc default/usb_specific_request.o
 .debug_info    0x000014a3      0x8eb default/usb_standard_request.o
 .debug_info    0x00001d8e      0x134 default/usb_task.o
 .debug_info    0x00001ec2       0xb9 default/stk_525.o
 .debug_info    0x00001f7b      0x1d0 default/hid_task.o
 .debug_info    0x0000214b      0x18e default/twimaster.o
 .debug_info    0x000022d9      0x107 default/scheduler.o
 *(.gnu.linkonce.wi.*)

.debug_abbrev   0x00000000      0x9a2
 *(.debug_abbrev)
 .debug_abbrev  0x00000000       0x7b default/wdt_drv.o
 .debug_abbrev  0x0000007b       0xc2 default/usb_descriptors.o
 .debug_abbrev  0x0000013d       0x71 default/usb_device_task.o
 .debug_abbrev  0x000001ae       0xbf default/usb_drv.o
 .debug_abbrev  0x0000026d       0x69 default/start_boot.o
 .debug_abbrev  0x000002d6       0x73 default/main.o
 .debug_abbrev  0x00000349      0x1be default/usb_specific_request.o
 .debug_abbrev  0x00000507      0x20d default/usb_standard_request.o
 .debug_abbrev  0x00000714       0x86 default/usb_task.o
 .debug_abbrev  0x0000079a       0x2a default/stk_525.o
 .debug_abbrev  0x000007c4       0xcb default/hid_task.o
 .debug_abbrev  0x0000088f       0xba default/twimaster.o
 .debug_abbrev  0x00000949       0x59 default/scheduler.o

.debug_line     0x00000000     0x21d2
 *(.debug_line)
 .debug_line    0x00000000      0x203 default/wdt_drv.o
 .debug_line    0x00000203      0x14d default/usb_descriptors.o
 .debug_line    0x00000350      0x2c3 default/usb_device_task.o
 .debug_line    0x00000613      0x289 default/usb_drv.o
 .debug_line    0x0000089c      0x17c default/start_boot.o
 .debug_line    0x00000a18      0x163 default/main.o
 .debug_line    0x00000b7b      0x5b7 default/usb_specific_request.o
 .debug_line    0x00001132      0x5d4 default/usb_standard_request.o
 .debug_line    0x00001706      0x2c7 default/usb_task.o
 .debug_line    0x000019cd       0xea default/stk_525.o
 .debug_line    0x00001ab7      0x313 default/hid_task.o
 .debug_line    0x00001dca      0x26a default/twimaster.o
 .debug_line    0x00002034      0x19e default/scheduler.o

.debug_frame    0x00000000      0x3e0
 *(.debug_frame)
 .debug_frame   0x00000000       0x50 default/wdt_drv.o
 .debug_frame   0x00000050       0x40 default/usb_device_task.o
 .debug_frame   0x00000090       0x70 default/usb_drv.o
 .debug_frame   0x00000100       0x40 default/start_boot.o
 .debug_frame   0x00000140       0x30 default/main.o
 .debug_frame   0x00000170       0xc0 default/usb_specific_request.o
 .debug_frame   0x00000230       0x30 default/usb_standard_request.o
 .debug_frame   0x00000260       0x40 default/usb_task.o
 .debug_frame   0x000002a0       0x60 default/hid_task.o
 .debug_frame   0x00000300       0x90 default/twimaster.o
 .debug_frame   0x00000390       0x50 default/scheduler.o

.debug_str      0x00000000      0xc98
 *(.debug_str)
 .debug_str     0x00000000      0x194 default/wdt_drv.o
                                0x1e5 (size before relaxing)
 .debug_str     0x00000194      0x3b4 default/usb_descriptors.o
                                0x526 (size before relaxing)
 .debug_str     0x00000548       0xbd default/usb_device_task.o
                                0x215 (size before relaxing)
 .debug_str     0x00000605       0xda default/usb_drv.o
                                0x232 (size before relaxing)
 .debug_str     0x000006df       0x69 default/start_boot.o
                                0x1c1 (size before relaxing)
 .debug_str     0x00000748       0x28 default/main.o
                                0x180 (size before relaxing)
 .debug_str     0x00000770      0x1d5 default/usb_specific_request.o
                                0x644 (size before relaxing)
 .debug_str     0x00000945      0x199 default/usb_standard_request.o
                                0x644 (size before relaxing)
 .debug_str     0x00000ade       0x43 default/usb_task.o
                                0x1d2 (size before relaxing)
 .debug_str     0x00000b21       0x25 default/stk_525.o
                                0x17d (size before relaxing)
 .debug_str     0x00000b46       0x70 default/hid_task.o
                                0x1ed (size before relaxing)
 .debug_str     0x00000bb6       0x74 default/twimaster.o
                                0x181 (size before relaxing)
 .debug_str     0x00000c2a       0x6e default/scheduler.o
                                0x1c6 (size before relaxing)

.debug_loc      0x00000000      0x90c
 *(.debug_loc)
 .debug_loc     0x00000000       0x5a default/wdt_drv.o
 .debug_loc     0x0000005a      0x122 default/usb_drv.o
 .debug_loc     0x0000017c      0x2c3 default/usb_specific_request.o
 .debug_loc     0x0000043f      0x3f0 default/usb_standard_request.o
 .debug_loc     0x0000082f       0x1e default/hid_task.o
 .debug_loc     0x0000084d       0xbf default/twimaster.o

.debug_macinfo
 *(.debug_macinfo)
OUTPUT(USBKEY_STK525-series6-hidio.elf elf32-avr)
LOAD linker stubs

.debug_ranges   0x00000000       0x30
 .debug_ranges  0x00000000       0x30 default/usb_standard_request.o

Cross Reference Table

Symbol                                            File
__bad_interrupt                                   c:/winavr/bin/../lib/gcc/avr/4.1.1/../../../../avr/lib/avr5/crtusb1286.o
__bss_end                                         c:/winavr/bin/../lib/gcc/avr/4.1.1/avr5\libgcc.a(_clear_bss.o)
__bss_start                                       c:/winavr/bin/../lib/gcc/avr/4.1.1/avr5\libgcc.a(_clear_bss.o)
__data_end                                        c:/winavr/bin/../lib/gcc/avr/4.1.1/../../../../avr/lib/avr5/crtusb1286.o
__data_load_start                                 c:/winavr/bin/../lib/gcc/avr/4.1.1/../../../../avr/lib/avr5/crtusb1286.o
__data_start                                      c:/winavr/bin/../lib/gcc/avr/4.1.1/../../../../avr/lib/avr5/crtusb1286.o
__do_clear_bss                                    c:/winavr/bin/../lib/gcc/avr/4.1.1/avr5\libgcc.a(_clear_bss.o)
                                                  default/scheduler.o
                                                  default/twimaster.o
                                                  default/hid_task.o
                                                  default/stk_525.o
                                                  default/usb_task.o
                                                  default/usb_standard_request.o
                                                  default/usb_specific_request.o
                                                  default/main.o
                                                  default/start_boot.o
                                                  default/usb_drv.o
                                                  default/usb_device_task.o
                                                  default/usb_descriptors.o
                                                  default/wdt_drv.o
__do_copy_data                                    c:/winavr/bin/../lib/gcc/avr/4.1.1/../../../../avr/lib/avr5/crtusb1286.o
                                                  default/scheduler.o
                                                  default/twimaster.o
                                                  default/hid_task.o
                                                  default/stk_525.o
                                                  default/usb_task.o
                                                  default/usb_standard_request.o
                                                  default/usb_specific_request.o
                                                  default/main.o
                                                  default/start_boot.o
                                                  default/usb_drv.o
                                                  default/usb_device_task.o
                                                  default/usb_descriptors.o
                                                  default/wdt_drv.o
__heap_end                                        c:/winavr/bin/../lib/gcc/avr/4.1.1/../../../../avr/lib/avr5/crtusb1286.o
__init                                            c:/winavr/bin/../lib/gcc/avr/4.1.1/../../../../avr/lib/avr5/crtusb1286.o
__low_level_init                                  default/main.o
__stack                                           c:/winavr/bin/../lib/gcc/avr/4.1.1/../../../../avr/lib/avr5/crtusb1286.o
__vector_1                                        c:/winavr/bin/../lib/gcc/avr/4.1.1/../../../../avr/lib/avr5/crtusb1286.o
__vector_10                                       default/usb_task.o
                                                  c:/winavr/bin/../lib/gcc/avr/4.1.1/../../../../avr/lib/avr5/crtusb1286.o
__vector_11                                       c:/winavr/bin/../lib/gcc/avr/4.1.1/../../../../avr/lib/avr5/crtusb1286.o
__vector_12                                       c:/winavr/bin/../lib/gcc/avr/4.1.1/../../../../avr/lib/avr5/crtusb1286.o
__vector_13                                       c:/winavr/bin/../lib/gcc/avr/4.1.1/../../../../avr/lib/avr5/crtusb1286.o
__vector_14                                       c:/winavr/bin/../lib/gcc/avr/4.1.1/../../../../avr/lib/avr5/crtusb1286.o
__vector_15                                       c:/winavr/bin/../lib/gcc/avr/4.1.1/../../../../avr/lib/avr5/crtusb1286.o
__vector_16                                       c:/winavr/bin/../lib/gcc/avr/4.1.1/../../../../avr/lib/avr5/crtusb1286.o
__vector_17                                       c:/winavr/bin/../lib/gcc/avr/4.1.1/../../../../avr/lib/avr5/crtusb1286.o
__vector_18                                       c:/winavr/bin/../lib/gcc/avr/4.1.1/../../../../avr/lib/avr5/crtusb1286.o
__vector_19                                       c:/winavr/bin/../lib/gcc/avr/4.1.1/../../../../avr/lib/avr5/crtusb1286.o
__vector_2                                        c:/winavr/bin/../lib/gcc/avr/4.1.1/../../../../avr/lib/avr5/crtusb1286.o
__vector_20                                       c:/winavr/bin/../lib/gcc/avr/4.1.1/../../../../avr/lib/avr5/crtusb1286.o
__vector_21                                       c:/winavr/bin/../lib/gcc/avr/4.1.1/../../../../avr/lib/avr5/crtusb1286.o
__vector_22                                       c:/winavr/bin/../lib/gcc/avr/4.1.1/../../../../avr/lib/avr5/crtusb1286.o
__vector_23                                       c:/winavr/bin/../lib/gcc/avr/4.1.1/../../../../avr/lib/avr5/crtusb1286.o
__vector_24                                       c:/winavr/bin/../lib/gcc/avr/4.1.1/../../../../avr/lib/avr5/crtusb1286.o
__vector_25                                       c:/winavr/bin/../lib/gcc/avr/4.1.1/../../../../avr/lib/avr5/crtusb1286.o
__vector_26                                       c:/winavr/bin/../lib/gcc/avr/4.1.1/../../../../avr/lib/avr5/crtusb1286.o
__vector_27                                       c:/winavr/bin/../lib/gcc/avr/4.1.1/../../../../avr/lib/avr5/crtusb1286.o
__vector_28                                       c:/winavr/bin/../lib/gcc/avr/4.1.1/../../../../avr/lib/avr5/crtusb1286.o
__vector_29                                       c:/winavr/bin/../lib/gcc/avr/4.1.1/../../../../avr/lib/avr5/crtusb1286.o
__vector_3                                        c:/winavr/bin/../lib/gcc/avr/4.1.1/../../../../avr/lib/avr5/crtusb1286.o
__vector_30                                       c:/winavr/bin/../lib/gcc/avr/4.1.1/../../../../avr/lib/avr5/crtusb1286.o
__vector_31                                       c:/winavr/bin/../lib/gcc/avr/4.1.1/../../../../avr/lib/avr5/crtusb1286.o
__vector_32                                       c:/winavr/bin/../lib/gcc/avr/4.1.1/../../../../avr/lib/avr5/crtusb1286.o
__vector_33                                       c:/winavr/bin/../lib/gcc/avr/4.1.1/../../../../avr/lib/avr5/crtusb1286.o
__vector_34                                       c:/winavr/bin/../lib/gcc/avr/4.1.1/../../../../avr/lib/avr5/crtusb1286.o
__vector_35                                       c:/winavr/bin/../lib/gcc/avr/4.1.1/../../../../avr/lib/avr5/crtusb1286.o
__vector_36                                       c:/winavr/bin/../lib/gcc/avr/4.1.1/../../../../avr/lib/avr5/crtusb1286.o
__vector_37                                       c:/winavr/bin/../lib/gcc/avr/4.1.1/../../../../avr/lib/avr5/crtusb1286.o
__vector_4                                        c:/winavr/bin/../lib/gcc/avr/4.1.1/../../../../avr/lib/avr5/crtusb1286.o
__vector_5                                        c:/winavr/bin/../lib/gcc/avr/4.1.1/../../../../avr/lib/avr5/crtusb1286.o
__vector_6                                        c:/winavr/bin/../lib/gcc/avr/4.1.1/../../../../avr/lib/avr5/crtusb1286.o
__vector_7                                        c:/winavr/bin/../lib/gcc/avr/4.1.1/../../../../avr/lib/avr5/crtusb1286.o
__vector_8                                        c:/winavr/bin/../lib/gcc/avr/4.1.1/../../../../avr/lib/avr5/crtusb1286.o
__vector_9                                        c:/winavr/bin/../lib/gcc/avr/4.1.1/../../../../avr/lib/avr5/crtusb1286.o
__vector_default                                  c:/winavr/bin/../lib/gcc/avr/4.1.1/../../../../avr/lib/avr5/crtusb1286.o
__vectors                                         c:/winavr/bin/../lib/gcc/avr/4.1.1/../../../../avr/lib/avr5/crtusb1286.o
boot_key                                          default/start_boot.o
cpt_sof                                           default/hid_task.o
data_to_transfer                                  default/usb_standard_request.o
                                                  default/usb_specific_request.o
endpoint_status                                   default/usb_standard_request.o
g_last_joy                                        default/hid_task.o
g_u8_report_rate                                  default/usb_specific_request.o
g_usb_event                                       default/usb_task.o
                                                  default/usb_device_task.o
goto_boot                                         default/start_boot.o
hid_get_hid_descriptor                            default/usb_specific_request.o
hid_get_report_descriptor                         default/usb_specific_request.o
hid_report_in                                     default/hid_task.o
hid_report_out                                    default/hid_task.o
hid_task                                          default/hid_task.o
                                                  default/scheduler.o
hid_task_init                                     default/hid_task.o
                                                  default/scheduler.o
i2c_init                                          default/twimaster.o
                                                  default/hid_task.o
i2c_readAck                                       default/twimaster.o
i2c_readNak                                       default/twimaster.o
i2c_rep_start                                     default/twimaster.o
i2c_start                                         default/twimaster.o
                                                  default/hid_task.o
i2c_start_wait                                    default/twimaster.o
i2c_stop                                          default/twimaster.o
                                                  default/hid_task.o
i2c_write                                         default/twimaster.o
                                                  default/hid_task.o
jump_bootloader                                   default/usb_specific_request.o
                                                  default/hid_task.o
main                                              default/main.o
                                                  c:/winavr/bin/../lib/gcc/avr/4.1.1/../../../../avr/lib/avr5/crtusb1286.o
pbuffer                                           default/usb_standard_request.o
                                                  default/usb_specific_request.o
remote_wakeup_feature                             default/usb_standard_request.o
                                                  default/usb_task.o
                                                  default/usb_device_task.o
ret                                               default/hid_task.o
                                                  default/main.o
scheduler                                         default/scheduler.o
                                                  default/main.o
scheduler_empty_fct                               default/scheduler.o
scheduler_init                                    default/scheduler.o
scheduler_tasks                                   default/scheduler.o
sof_action                                        default/hid_task.o
                                                  default/usb_task.o
start_boot                                        default/start_boot.o
                                                  default/hid_task.o
start_boot_if_required                            default/start_boot.o
                                                  default/main.o
start_bootloader                                  default/start_boot.o
usb_conf_desc                                     default/usb_descriptors.o
                                                  default/usb_standard_request.o
                                                  default/usb_specific_request.o
usb_config_ep                                     default/usb_drv.o
                                                  default/usb_specific_request.o
usb_configuration_nb                              default/hid_task.o
                                                  default/usb_task.o
                                                  default/usb_standard_request.o
                                                  default/usb_device_task.o
usb_connected                                     default/usb_device_task.o
usb_dev_desc                                      default/usb_descriptors.o
                                                  default/usb_standard_request.o
usb_device_task                                   default/usb_device_task.o
                                                  default/usb_task.o
usb_device_task_init                              default/usb_device_task.o
                                                  default/usb_task.o
usb_generate_remote_wakeup                        default/usb_standard_request.o
usb_halt_endpoint                                 default/usb_drv.o
usb_hid_get_idle                                  default/usb_specific_request.o
usb_hid_report_descriptor                         default/usb_descriptors.o
                                                  default/usb_specific_request.o
usb_hid_set_idle                                  default/usb_specific_request.o
usb_hid_set_report_feature                        default/usb_specific_request.o
usb_hid_set_report_ouput                          default/usb_specific_request.o
usb_init_device                                   default/usb_drv.o
                                                  default/usb_task.o
                                                  default/usb_device_task.o
usb_process_request                               default/usb_standard_request.o
                                                  default/usb_device_task.o
usb_read_packet                                   default/usb_drv.o
usb_select_enpoint_interrupt                      default/usb_drv.o
usb_send_packet                                   default/usb_drv.o
usb_start_device                                  default/usb_device_task.o
usb_suspended                                     default/usb_device_task.o
usb_task                                          default/usb_task.o
                                                  default/scheduler.o
usb_task_init                                     default/usb_task.o
                                                  default/scheduler.o
usb_user_endpoint_init                            default/usb_specific_request.o
                                                  default/usb_standard_request.o
usb_user_get_descriptor                           default/usb_specific_request.o
                                                  default/usb_standard_request.o
usb_user_interface_get                            default/usb_specific_request.o
                                                  default/usb_standard_request.o
usb_user_interface_reset                          default/usb_specific_request.o
                                                  default/usb_standard_request.o
usb_user_language_id                              default/usb_descriptors.o
                                                  default/usb_specific_request.o
usb_user_manufacturer_string_descriptor           default/usb_descriptors.o
                                                  default/usb_specific_request.o
usb_user_product_string_descriptor                default/usb_descriptors.o
                                                  default/usb_specific_request.o
usb_user_read_request                             default/usb_specific_request.o
                                                  default/usb_standard_request.o
wdtdrv_disable                                    default/wdt_drv.o
                                                  default/main.o
wdtdrv_enable                                     default/wdt_drv.o
                                                  default/start_boot.o
wdtdrv_interrupt_enable                           default/wdt_drv.o
wdtdrv_interrupt_reset_enable                     default/wdt_drv.o
